:04000000B601CD294F
:100008000800B616B61EB612B6190E28B615472041
:10001800031835280830A3005B20A20DA30B102875
:10002800B61E402065206120B61A35203A202208E5
:100038000310C829B616B61EB61236192828FE3976
:10004800B70036150310C829361A3028A600361608
:1000580047200318352826084E2003183528B61ED1
:10006800C8294020652036113612B6113A08840096
:1000780038088417800446283A088400380980051F
:100088008417800508003A20652040206120370841
:10009800B6190138A2000830A300A20D03183A20AF
:1000A800031C402065206120A30B51283A206520BD
:1000B8003A08840038080005FF3E3B0884003909E7
:1000C80043283B08840039083D2864007F20031832
:1000D8006928CE20A8010830A300CF207F2003186C
:1000E800A80AAB1EA801A20CA30B7128AB1AA21375
:1000F800CF20220808003A088400380884178004B2
:10010800841300052B1B3806FF3E0800A4002908AD
:100118000319C829C321A0002518831724088400BF
:10012800200880008313A40AA9038B280408A600CA
:100138003A088400F030B7050830A7000310031808
:10014800B70AB420A60CA70BA3280000AB1A370CDB
:10015800B420CB210314B4202F08A3002E082F2984
:100168008413AB1FC328000838042B1F38068000EF
:10017800841700083804031C38068000CF280008BC
:100188003804031C38062B1B3806800084173809EE
:100198008005CF2837172B081F39003EA1002A08F1
:1001A8000E3E0318A10A371F3C293713A00002305E
:1001B80060213C29B71329080319B7170430A80090
:1001C800250EEB202508EB20240EEB2024080F3900
:1001D800F63E0318073E0A3EF128A000A8030319BB
:1001E800B71329080319FB28280203180800200858
:1001F800031DB713B71B0800303EC32983178001BE
:10020800840AFF3E031D0329C82921082004031975
:10021800A00A8030201AA1062019A106A018A1065C
:10022800210DA00DA10DC82903178D0083168C136D
:100238000C1483120C08C82903178C0083168C131E
:100248000C1555308D00AA308D008C148C182A2975
:100258000C11C829A301A200FF30A207031CA307A1
:10026800031CC8290330A100E7303C213029A10133
:10027800FC3EA000A109031C4729FF300000A0078D
:1002880003184229A0076400A10F41290800013E74
:10029800A7000A30A200A3019121A70B5029240826
:1002A80008000310A00DA10DFF3E031855292008D2
:1002B800C8290310A10CA00CFF3E03185D292008D3
:1002C800C829A101A301A20002307A29A301A20032
:1002D80003307A29A301A20001307A29A301A200E0
:1002E80006307A29A101A301A2000530A80023083D
:1002F8002102031D8129220820020430031801303D
:10030800031902302805031DFF30C8290038031DD2
:10031800FF300405031DFF30C8291030A600A501D1
:10032800A401210DA40DA50D2208A4022308031C75
:10033800230FA5020318A7292208A40723080318D6
:10034800230FA5070310A00DA10DA60B95292008C2
:10035800C8291030A800A101A001A70CA60C031CF5
:10036800BB292208A00723080318230FA107A10C03
:10037800A00CA50CA40CA80BB1292408C82984003A
:1003880031088A0030088200831303138312640043
:1003980008002030840060308A010321A0308400E6
:1003A80050308A0103211030840060308A01022114
:1003B8009030840060308A010221831607309F0044
:1003C800990183129801831602309800EE01EF011B
:1003D800E301E20106108610061188018710071054
:1003E8000711871205128512DB01CE01C301013006
:1003F800CD00E801C430E700C201CE01C301E80125
:10040800C430E7008312880186140615871407157F
:10041800871207140130A300F4308A012F218316B4
:10042800DB01B0011030B100B401B50164005B0814
:10043800003C8A110A128312031D312A83160830E0
:10044800BA000730B9002030AE00AF012030B2004A
:10045800B30183128A110A123D2A83160630BA00A4
:100468000530B9002830AE00AF012830B200B30122
:100478008312071064308A012E2107148A150A1284
:10048800032B8A110A126C2283165C0883128800D7
:100498000711061587108610861487148A110A1208
:1004A8006C2283165D0883128800071106158710D1
:1004B8008610861487148A110A126C2283165A0829
:1004C8008312880006158710861086148714080082
:1004D80087148316FF308800831207158614871047
:1004E8000611003008180130A00001308A01762179
:1004F800B200003088180130A00001308A0176214E
:10050800B4003208840034088A018A218A110A1248
:10051800031D6C2A061587148316880183120800A8
:100528008A016C228316FF30880083120711061196
:10053800871002308A013B2108088316C000831205
:100548008714061583168801831208008A110A1277
:1005580050238A019422080083160130E800831290
:1005680083162A088312A60083162B088312A70075
:100578002030A200A3018A01AD21B2002508B300F2
:10058800831630088312B207831631080318013E18
:100598008312B307831628088312A000831629083C
:1005A8008312A10083163A088312A200A3018A01CC
:1005B8009121B4002108B500320834078316A00041
:1005C800831233080318013E35078316A10020085B
:1005D800A6002108A7002808CB002A08CC0021087B
:1005E800DD002008DC002430DA0083128A0145226D
:1005F800640083166808003C8A110A128312031DDE
:10060800292B831628088312A00083162908831231
:10061800A10083163A088312A200A3018A0191213E
:100628002408B2002508B300320883163902831261
:10063800B20033090318013EB300F83032048316C0
:10064800DA0083128A110A124A2B831628088312A9
:10065800A000831629088312A10083163A08831282
:10066800A200A3018A0191212408B2002508B30041
:100678003208831639028312B20033090318013E87
:10068800B300F03032048316DA0083128A015F2245
:100698008316E8018312080083162A088312A6002D
:1006A80083162B088312A7002030A200A3018A0119
:1006B800AD21B2002508B300831630088312B207B3
:1006C800831631080318013E8312B30783162808DE
:1006D8008312A000831629088312A10083163A0802
:1006E8008312A200A3018A019121B4002108B50058
:1006F800320834078316A000831233080318013E1A
:1007080035078316A1002008A6002108A7002108A4
:10071800DD002008DC002430DA0083128A0145223B
:100728000800831658085507A800A901A90D5908FB
:100738005607AA00AB01AB0D83128A01B4228316B7
:1007480058085502A800A901031CA903590856070F
:10075800AA00AB01AB0D83128A01B4228316550897
:100768005807A800A901A90D59085602AA00AB010B
:10077800031CAB0383128A01B4228316580855025E
:10078800A800A901031CA90359085602AA00AB0135
:10079800031CAB0383128A01B42283165908550738
:1007A800A800A901A90D58085607AA00AB01AB0D6E
:1007B80083128A01B422831659085502A800A90198
:1007C800031CA90356085807AA00AB01AB0D8312F6
:1007D8008A01B422831655085907A800A901A90D52
:1007E80058085602AA00AB01031CAB0383128A0106
:1007F800B422831659085502A800A901031CA903AD
:1008080058085602AA00AB01031CAB0383128A01E5
:10081800B422080083163108DD003008DC004230BD
:10082800DA0083128A01452283162F08DD002E087C
:10083800DC004330DA0083128A014522831635082A
:10084800DD003408DC004030DA0083128A014522DA
:1008580083163308DD003208DC004130DA008312E9
:100868008A01452283168030DA0083128A015F22CA
:100878008316DD01DC012430DA0083128A01452267
:1008880083169830DA0083128A015F2283160130BA
:10089800C30083126400F130831643028A110A12DE
:1008A80083120318792C83160130C6008312640062
:1008B8004130831646028A110A1283120318722CD9
:1008C8008316DD01C030DA0083128A0152228316B2
:1008D800C60A8A110A128312031D5B2C8316C30AE7
:1008E8008A110A128312031D4E2C83169C30DA00DB
:1008F80083128A015F2208008316D8015708D9009D
:100908000310570D8312B200B301B30D3208023C35
:100918008316AC0083123308031C013E003C831687
:10092800AD00831264008316580859028A110A120E
:100938008312031CF12C8A01952364008A110A1280
:1009480083168310AD1F831483128318C92C0430B7
:10095800A600A701831658088312A200A3018A01E2
:10096800AD21B2002508B3000630B2070318B30A58
:1009780032088316AC07831233080318013E831626
:10098800AD0783128A110A12EC2C831659085802F3
:100998008312B200B301031CB3030430A600A701FD
:1009A8003208A2003308A3008A01AD21B20025084D
:1009B800B3000A30B2070318B30A32088316AC072B
:1009C800831233080318013E8316AD07D903831237
:1009D8008316D80A83128A01962C08008316D80138
:1009E8005708D9000310570D8312B200B301B30D95
:1009F8003208023C8316AC0083123308031C013E04
:100A0800003C8316AD00831264008316580859020F
:100A18008A110A128312031C3A2D8A019523831620
:100A2800590858028312B200B301031CB3030430FF
:100A3800A600A7013208A2003308A3008A01AD214D
:100A4800B2002508B3000A30B2070318B30A320807
:100A58008316AC07831233080318013E8316AD07CB
:100A68000330D902D80A83128A01082D08008A1196
:100A78000A123B2683164F085002C8005208530238
:100A8800C9006400490848028A110A128312031C2B
:100A9800C42D831649088312A000A10102308A01DF
:100AA8005821B2002108B300831648088312320285
:100AB8008316AC0083123308031CFF3E8316AD0077
:100AC8005208AA00AB0149088312A000A101023014
:100AD8008A0158218316A200831221088316A300D5
:100AE800480849028312B200B301031CB303031080
:100AF800320D8316A4008312330D8316A5004F0808
:100B0800A800A9018312831628088312A00083165F
:100B180029088312A1008316500883128A016E21C6
:100B28008A110A12031DC32D64008A110A12831642
:100B38008310AD1F831483128318AD2D83162208EA
:100B4800AC0723080318013EAD0783128A110A1265
:100B5800B82D83162408AC0725080318013EAD07F5
:100B6800AA0A0319AB0A83128A01B4228316A80AB7
:100B78000319A90A8A110A128312031D872D080076
:100B8800831648088312A000A10102308A01582167
:100B9800B2002108B3008316490883123202831673
:100BA800AC0083123308031CFF3E8316AD004F08C8
:100BB800A800A90148088312A000A10102308A01F7
:100BC80058218316A200831221088316A30049081E
:100BD80048028312B200B301031CB3030310320DA1
:100BE8008316A4008312330D8316A5005208AA00A9
:100BF800AB01831283162A088312A00083162B08E0
:100C08008312A1008316530883128A016E218A1168
:100C18000A12031D3A2E64008A110A1283168310E1
:100C2800AD1F831483128318242E83162208AC0761
:100C380023080318013EAD0783128A110A122F2ECA
:100C480083162408AC0725080318013EAD07A80A37
:100C58000319A90A83128A01B4228316AA0A03195E
:100C6800AB0A8A110A128312031DFE2D08006400C4
:100C780083164F0850028A110A12831203184A2E4B
:100C880083164F085002CF07D002831264008316E0
:100C9800520853028A110A1283120318592E831616
:100CA80052085302D207D3028312080083162A0877
:100CB8008312A00083162B088312A1000830A2001B
:100CC800A3018A019121B2002108B3003208A600CD
:100CD8003308A7002030A200A3018A01AD21B20089
:100CE8002508B300831634088312B2078316350823
:100CF8000318013E8312B307831628088312A00045
:100D0800831629088312A10083163A088312A200C9
:100D1800A3018A019121B4002108B50032083407E3
:100D28008316A000831233080318013E3507831683
:100D3800A1002108DD002008DC002430DA0083123D
:100D48008A01452208008A110A12B5278A0145221C
:100D58008A110A126227203083163B02BF008312D1
:100D68008A015A2683163F08DD006708DA008312D5
:100D78008A0152228A110A126C2708007D08A000F5
:100D88007E08A10004308A014B218316BB00831220
:100D98008A110A121C2708308316A8070318A90A03
:100DA80083127D08A0007E08A10003308A014B2130
:100DB8008316BB0083128A110A121C270830831677
:100DC800A8070318A90A83127D08A0007E08A100BD
:100DD80002308A014B218316BB0083128A110A1242
:100DE8001C2708308316A8070318A90A83127D0850
:100DF800A0007E08A10001308A014B218316BB00A8
:100E080083128A110A121C2708308316A8070318B0
:100E1800A90A83127D08A0007E08A10000308A017B
:100E28004B218316BB0083128A110A121C27080063
:100E380083163B08093C8A110A128312031C3D2FB2
:100E48008A110A122D278316CE0083128A110A12DC
:100E58003D2F07308A0083163B08831282073034FF
:100E68003134323433343434353436343734383436
:100E78003934203083164E02BF0083128A01B4260B
:100E880008008A110A12B5278A110A1262278A01F4
:100E9800502383163E08DD006708DA0083128A01B2
:100EA80052228A110A126C2708008A0145228316E9
:100EB8009830DA0083128A015F2208008A110A1228
:100EC800B52783169430DA0083128A015F2208005E
:100ED8008A110A12B52783169C30DA0083128A0118
:100EE8005F220800831643085C3E840000088312D2
:100EF800B200FF30A200A20A22080F3C8A110A128F
:100F0800031CA92F8A110A12952732028A110A1284
:100F1800031D7F2F22088316DE0083128A110A120E
:100F2800A92F07308A00220882073034313432343E
:100F3800333434343534363437343834393461342E
:100F480062346334643465346634080083163108C7
:100F5800DD003008DC004230DA0083128A014522C5
:100F6800080083163508DD003408DC004030DA005C
:100F780083128A014522080083166B08A800A9017C
:100F88006D08AA00AB01831283162A088312A000F9
:100F980083162B088312A10083166C0883128A011A
:100FA8006E218A110A12031DE42F8A01B4228316C6
:100FB800AA0A0319AB0A8A110A128312031DC82F41
:100FC800013083166B07A800A901A90D6D08AA00B6
:100FD800AB01831283162A088312A00083162B08FC
:100FE8008312A10083166C0883128A016E218A1568
:100FF8000A12031D10288A01B42283166908AA0759
:101008008A110A128312031CEE2F8316AA0A8A1168
:101018000A128312031DEE2F080083166D08AA001A
:10102800AB016B08A800A901831283162808831254
:10103800A000831629088312A10083166A08831268
:101048008A016E218A150A12031D35288A01B422E5
:101058008316A80A0319A90A8A150A128312031DFE
:101068001928FF3083166D07AA00FF300318013EC8
:10107800AB006B08A800A901831283162808831205
:10108800A000831629088312A10083166A08831218
:101098008A016E218A150A12031D63288A01B42267
:1010A80083166908A8078A150A128312031C4128A7
:1010B8008316A80A8A150A128312031D41280800FC
:1010C8008A013B2683164F08C300831264008316E7
:1010D800430850028A150A128312031C9A288316A1
:1010E8005208C600831264008316460853028A1504
:1010F8000A128312031C922883164308A800A90128
:101108004608AA00AB0183128A01B4228316690833
:10111800C6078A150A128312031C772883166908E2
:10112800C3078A150A128312031C6A2808008A0159
:101138003B2683164F08C3008312640083164308B6
:1011480050028A150A128312031CC3288316430807
:10115800A800A9015208AA00AB0183128A01B4228F
:1011680083165308AA00AB0183128A01B42283169E
:101178006908C3078A150A128312031CA12883165B
:101188005208C300831264008316430853028A1569
:101198000A128312031CE92883164308AA00AB012C
:1011A8004F08A800A90183128A01B42283165008A7
:1011B800A800A90183128A01B42283166908C3070B
:1011C8008A150A128312031CC72808008316D8013F
:1011D8005708D9000310570D8312B200B301B30D9D
:1011E8003208023C8316AC0083123308031C013E0C
:1011F800003C8316AD008312640083165808590218
:101208008A150A128312031C32298A019523831630
:10121800590858028312B200B301031CB303043007
:10122800A600A7013208A2003308A3008A01AD2155
:10123800B2002508B3000A30B2070318B30A32080F
:101248008316AC07831233080318013E8316AD07D3
:10125800D903D80A83128A150A12002908008316AE
:10126800D8015708D9000310570D8312B200B301F3
:10127800B30D3208023C8316AC0083123308031CFA
:10128800013E003C8316AD008312640083165808A3
:1012980059028A150A128312031C73298A0195239D
:1012A8000430A600A701831658088312A200A301E0
:1012B8008A01AD21B2002508B3000630B207031831
:1012C800B30A32088316AC07831233080318013EA9
:1012D8008316AD07D80A83128A150A12492908000D
:1012E8000730BA004030B8002030AA00AB01AE0188
:1012F800AF010230A900831640088312A400A5019B
:101308009A30B000B1018A01DE2008000730BA0027
:101318008030B8002030AA00AB018A0169205D3C0A
:101328008A150A12031D91290230A9006930B000FC
:10133800B101A5015C308A018A208316C30183129A
:1013480064000230831643028A150A1283120318B6
:10135800BB298A017627831643085C3E84005E0811
:101368008000C30A8A150A128312031DA4295C0887
:10137800A000A10104308A015821B2002108B3005D
:101388005D083204FF0008000730BA008030B8005A
:101398002030AA00AB018A0169205D3C8A150A1237
:1013A800031DCF290430A9006930B000B101A5019F
:1013B8005C308A018A208316C301831264000430DA
:1013C800831643028A150A1283120318F9298A011F
:1013D8007627831643085C3E84005E088000C30AB3
:1013E8008A150A128312031DE2295C08A000A101D4
:1013F80004308A015821B2002108B3005D08320484
:10140800FF005E08A000A10104308A015821B20043
:101418002108B3005F0832048316B600831208005F
:101428000730BA008030B8002030AA00AB018A012A
:1014380069205D3C8A150A12031D1B2A0630A90083
:101448006930B000B101A5015C308A018A20831699
:10145800C301831264000630831643028A150A12F8
:1014680083120318452A8A017627831643085C3EAF
:1014780084005E088000C30A8A150A128312031DBD
:101488002E2A5C08A000A10104308A015821B2006C
:101498002108B3005D083204FF005E08A000A10126
:1014A80004308A015821B2002108B3005F083204D1
:1014B8008316B60083126008A000A10104308A01D7
:1014C8005821B2002108B300610832048316B7001E
:1014D800831208000730BA008030B8002030AA0014
:1014E800AB018A0169205D3C8A150A12031D752A21
:1014F8008A0169208316DE0030305E02E9005E084A
:10150800C000831208000730BA008030B8002030CD
:10151800AA00AB018A0169205D3C8A150A12031DE5
:101528008E2A0830A9006930B000B101A5015C30ED
:101538008A018A208316C301831264000830831647
:1015480043028A150A1283120318B82A8A017627D9
:10155800831643085C3E84005E088000C30A8A152F
:101568000A128312031DA12A5C08A000A1010430FD
:101578008A015821B2002108B3005D08320483169D
:10158800CF0083125E08A000A10104308A0158210F
:10159800B2002108B3005F0832048316D00083121A
:1015A8006008A000A10104308A015821B200210876
:1015B800B300610832048316D20083126208A000C7
:1015C800A10104308A015821B2002108B300630840
:1015D80032048316D300831208007F088316D500CF
:1015E8003608D6003708D700831208007F0883160C
:1015F800A800A9013608AA00AB01831208008A01D5
:101608000E248A015927F901FA018316AA01AB01B0
:10161800831283162A088312A00083162B088312CC
:10162800A100A3013F308A016F218A150A12031D08
:10163800642B8316A801A901831283162808831234
:10164800A000831629088312A100A301EF308A01A4
:101658006F218A150A12031D5B2B0730BA00103060
:10166800B8000730BB000830B900A0308A0120203C
:101678007A088A01202079088A0120208A01052019
:101688008316BE0083128A014527F90A0319FA0A4C
:1016980008308316A8078A150A128312031C212B07
:1016A8008316A90A8A150A128312031D212B831691
:1016B800AA0A0319AB0A8A150A128312031D0D2BF5
:1016C80087140730A300D0308A012F218A013C24D7
:1016D8008A016C2783167730D5001F30D6000A3070
:1016E800D700831264001F30831657028A150A1226
:1016F80083120318892B8A0180240A308316D7079E
:101708008A150A128312031C762B83162D30D500F6
:101718001F30D6000A30D700831264001F308316AA
:1017280057028A150A1283120318A52B8A150A1262
:1017380033210A308316D7078A150A128312031C2D
:10174800912B8316C230D5001F30D6000A30D7003F
:10175800831264001F30831657028A150A128312F7
:101768000318C12B8A150A12EA200A308316D707F4
:101778008A150A128312031CAD2B0730A300D03040
:101788008A012F218A013C248A016C27831608309C
:10179800A800A9010830AA00AB01C30183126400A4
:1017A8001B30831643028A150A1283120318292C48
:1017B800831643081A3C8A150A128312031C1C2C30
:1017C8008A150A12ED238316BB0083128A150A12A2
:0E17D8001C2C0C308A00831643088312002C50
:101800008207533468346134723470342034323493
:1018100034343034783436343434203475347334DA
:1018200069346E34673420346134203454343634AF
:1018300039343634333443348A01A72608308316CA
:10184000A8070318A90AC30A8A150A128312031DDE
:10185000D32B0730A300D0308A012F218A150A121A
:10186000C62F83163030A800A9011830AA00AB019A
:10187000C301831264001530831643028A150A12CD
:10188000831203187C2C83164308143C8A150A1211
:101890008312031C6F2C8A150A1254248316BB0072
:1018A00083128A150A126F2C0C308A0083164308A3
:1018B0008312820753346F3466347434773461345E
:1018C0007234653420343234343420344A3475343C
:1018D0006E346534203432343034303431348A015B
:1018E000A72608308316A8070318A90AC30A8A1571
:1018F0000A128312031D3A2C83162230AA00AB0170
:101900003030A800A9018312831628088312A00092
:10191000831629088312A100A301D8308A016F2100
:101920008A150A12031DAB2C83162130AA00AB01C5
:1019300083128A01B42283162330AA00AB018312DA
:101940008A01B4228316A80A0319A90A8A150A1261
:101950008312031D842C0730A300D0308A012F216D
:101960008A010E248A016C2783160430E9000A30AC
:10197000ED003230EC000A30EB007830EA008312E0
:101980008A150A1211208A01C0278316A801A9010D
:101990001030AA00AB01C301831264000430831627
:1019A00043028A150A1283120318FE2C8316430879
:1019B000033C8A150A128312031CF12C8A150A12A1
:1019C000E7248316BB0083128A150A12F12C0C300F
:1019D0008A008316430883128207543445344D34F9
:1019E00050348A01A72608308316AA070318AB0AC9
:1019F000C30A8A150A128312031DCD2C83162030C8
:101A0000A800A9013830AA00AB01C3018312640009
:101A10000630831643028A150A12831203183A2DE0
:101A200083164308053C8A150A128312031C2D2DC8
:101A30008A150A1221258316BB0083128A150A1201
:101A40002D2D0D308A0083164308831282074834F7
:101A50004F34553452344C3459348A01A726083057
:101A60008316A8070318A90AC30A8A150A12831243
:101A7000031D072DFF3083166C07AA00FF300318E3
:101A8000013EAB006B08A800A90183128316280849
:101A90008312A000831629088312A10083166A0806
:101AA00083128A016E218A150A12031DBD2D831629
:101AB00022088312A000831623088312A1008A0142
:101AC000092120088316A200831221088316A3008F
:101AD0006400803022028A150A128312031C7B2DB7
:101AE00001308316AA020030031C013EAB028312B0
:101AF0008A150A12802D8316AA0A0319AB0A8312CB
:101B000083162A088312A00083162B088312A100D3
:101B100083166C0883128A0172218A150A12031D2A
:101B20009A2DFF3083166C07AA00FF300318013E80
:101B3000AB00831283162A088312A00083162B0899
:101B40008312A10083166D0883128A016A218A1507
:101B50000A12031DB22D013083166D07AA00AB01D6
:101B6000AB0D83128A01B4228316A80A0319A90AAD
:101B70008A150A128312031D462D83168230A8008F
:101B8000A9010830AA00AB01C3018312640006302A
:101B9000831643028A150A1283120318F92D83163D
:101BA0004308053C8A150A128312031CEC2D8A1582
:101BB0000A12E0258316BB0083128A150A12EC2D47
:101BC0000D308A00831643088312820743346F3432
:101BD00075346E3474343A348A01A726083083167B
:101BE000A8070318A90AC30A8A150A128312031D3B
:101BF000C62D83162030A800A901AA01AB01C3019C
:101C0000831264000730831643028A150A12831276
:101C10000318352E83164308063C8A150A128312D0
:101C2000031C282E8A150A121B268316BB0083125A
:101C30008A150A12282E0E308A0083164308831252
:101C400082074434493447344934563441344334A8
:101C50008A01A72608308316A8070318A90AC30A11
:101C60008A150A128312031D012E83168230A800E2
:101C7000A9011030AA00AB01C30183126400063031
:101C8000831643028A150A1283120318712E8316D3
:101C90004308053C8A150A128312031C642E8A1518
:101CA0000A1258268316BB0083128A150A12642E64
:101CB0000E308A008316430883128207203454347E
:101CC00065346D3470343A348A01A726083083169F
:101CD000A8070318A90AC30A8A150A128312031D4A
:101CE0003E2E83168230A800A9011830AA00AB014D
:101CF000C301831264000630831643028A150A1258
:101D000083120318AD2E83164308053C8A150A1268
:101D10008312031CA02E8A150A1294268316BB0078
:101D200083128A150A12A02E0E308A0083164308E9
:101D300083128207203454346F34723472343A344C
:101D40008A01A72608308316A8070318A90AC30A20
:101D50008A150A128312031D7A2E83168230A80078
:101D6000A9012030AA00AB01C30183126400063030
:101D7000831643028A150A1283120318E92E83166A
:101D80004308053C8A150A128312031CDC2E8A15AF
:101D90000A12D0268316BB0083128A150A12DC2E83
:101DA0000E308A0083164308831282075434693444
:101DB0006D3465344D343A348A01A72608308316D1
:101DC000A8070318A90AC30A8A150A128312031D59
:101DD000B62E83168230A800A9012830AA00AB01D4
:101DE000C301831264000630831643028A150A1267
:101DF00083120318252F83164308053C8A150A12FF
:101E00008312031C182F8A150A120C278316BB0095
:101E100083128A150A12182F0F308A00831643087E
:101E200083128207543469346D34653453343A3440
:101E30008A01A72608308316A8070318A90AC30A2F
:101E40008A150A128312031DF22E8316CE01831205
:101E5000FB01FC018316B430A800A9010830AA00D8
:101E6000AB018312FB0A0319FC0A7B08A0007C0863
:101E7000A100FF30A300FE308A0173218A150A12E7
:101E8000031D442FFB01FC017B08FD007C08FE00C4
:101E90008A01D5268316B430A800A9011030AA0003
:101EA000AB0183127D08A0007E08A10002308A01E8
:101EB0004B218316BB0083128A01B4260830831697
:101EC000A8070318A90A83127D08A0007E08A100B4
:101ED00001308A014B218316BB0083128A01B4268C
:101EE00008308316A8070318A90A83127D08A000EA
:101EF0007E08A10000308A014B218316BB008312AB
:101F00008A01B42608308316A8070318A90A2E30C0
:101F1000BB0083128A01A72608308316A80703187E
:101F2000A90A83127D08A0007E08A10000308A0162
:101F30004B218316BB0083128A01B4260830831616
:101F4000A8070318A90A4330BB0083128A01A726F9
:101F50008316B430A800A9011830AA00AB0183127F
:101F60008A010E278316B430A800A9012030AA00E8
:101F7000AB0183128A010E278316B430A800A90191
:101F80002830AA00AB0183128A01FB260730BA0071
:101F90004030B8002030AA00AB01AE01AF01523092
:101FA0008A019B2065308A019B2061308A019B2039
:101FB00064308A019B2079308A019B203A308A0163
:101FC0009B200A308A019B200D308A019B2007301C
:101FD000BA008030B8002030AA00AB018A01692025
:101FE0005D3C8A150A12031DEE2F8A0169208316B3
:101FF000DE005E088312A00063308A016521B20012
:1020000083165E088312A00043308A016521B40064
:10201000320834048A110A16031DF52983165E0856
:102020008312A00073308A016521B20083165E0816
:102030008312A00053308A016521B40032083404B1
:102040008A110A16031D002A83165E088312A00057
:1020500071308A016521B20083165E088312A000E8
:1020600051308A016521B400320834048A110A16FD
:10207000031D0C2A83165E088312A00074308A01A7
:102080006521B20083165E088312A00054308A01D5
:102090006521B400320834048A110A16031D182A77
:1020A00083165E088312A0006C308A016521B2009D
:1020B00083165E088312A0004C308A016521B400AB
:1020C000320834048A110A16031D3B2A83165E085F
:1020D0008312A00072308A016521B20083165E0867
:1020E0008312A00052308A016521B4003208340402
:1020F0008A110A16031D2F2A83165E088312A00078
:1021000062308A016521B20083165E088312A00046
:1021100042308A016521B400320834048A110A165B
:10212000031D232A83165E088312A0006B308A01E8
:102130006521B20083165E088312A0004B308A012D
:102140006521B400320834048A110A16031D6A2A74
:1021500083165E088312A00064308A016521B200F4
:1021600083165E088312A00044308A016521B40002
:10217000320834048A110A16031D732A83165E0876
:102180008312A00065308A016521B20083165E08C3
:102190008312A00045308A016521B400320834045E
:1021A0008A110A16031D6F2A83165E088312A00087
:1021B00070308A016521B20083165E088312A00088
:1021C00050308A016521B400320834048A110A169D
:1021D000031D812A83165E088312A00075308A01D0
:1021E0006521B20083165E088312A00055308A0173
:1021F0006521B400320834048A110A16031D932A9B
:1022000083165E088312A00078308A016521B2002F
:1022100083165E088312A00058308A016521B4003D
:10222000320834048A110A16031D432A83165E08F5
:102230008312A00079308A016521B20083165E08FE
:102240008312A00059308A016521B4003208340499
:102250008A110A16031D572A83165E088312A000EE
:1022600066308A016521B20083165E088312A000E1
:1022700046308A016521B400320834048A110A16F6
:10228000031DA22A83165E088312A00068308A010B
:102290006521B20083165E088312A00048308A01CF
:1022A0006521B400320834048A110A16031DB32ACA
:1022B00083165E088312A00076308A016521B20081
:1022C00083165E088312A00056308A016521B4008F
:1022D000320834048A110A16031D062B83165E0881
:1022E0008312A0006D308A016521B20083165E085A
:1022F0008312A0004D308A016521B40032083404F5
:102300008A110A16031D5B2C83165E088312A00037
:102310006E308A016521B20083165E088312A00028
:102320004E308A016521B400320834048A110A163D
:10233000031D122C83165E088312A0006F308A01E1
:102340006521B20083165E088312A0004F308A0117
:102350006521B400320834048A110A16031D6D2B5E
:1023600083165E088312A00061308A016521B200E5
:1023700083165E088312A00041308A016521B400F3
:10238000320834048A110A16031D732B83165E0863
:102390008312A00067308A016521B20083165E08AF
:1023A0008312A00047308A016521B400320834044A
:1023B0008A110A16031D662B83165E088312A0007D
:1023C00077308A016521B20083165E088312A0006F
:1023D00057308A016521B400320834048A110A1684
:1023E000031D5F2B8A150A12C62F8A150A121422A2
:1023F0008A150A12F1228A0180248A150A12C62F30
:102400008A150A1214228A150A12F1228A150A1252
:1024100033218A150A12C62F8A150A1214228A1528
:102420000A12F1228A150A12EA208A150A12C62F08
:102430008A150A1214228A150A12F1228A01F2243C
:102440008A150A12C62F8A150A1287228A150A12BD
:102450006E228A150A1264208A150A12C62F8A155E
:102460000A1287228A150A126E228A150A129B20E6
:102470008A150A12C62F8A150A1287228A013B255D
:102480008A150A12C62F8A150A1214227F0883168B
:10249000EB003608EA003708ED0083128A150A12AD
:1024A0006E228A150A1211208A150A12C62F8A1561
:1024B0000A1214227F088316ED003608EC00370854
:1024C000EB0083128A150A126E228A01C0278A1530
:1024D0000A12C62F8A013C248A150A12C62F8316B7
:1024E0000130E80083128A150A12C8218A150A12DF
:1024F000FA228A01B4228316E80183128A150A128D
:10250000C62F8A150A12C8218A150A12FA228A15BC
:102510000A126E2283164008BB0083128A01A72686
:102520008A150A12C62F8A150A1214228A150A124F
:10253000FA2283163708BE0083128A0145278A15BE
:102540000A12C62F8A150A126E228316CF01EF30A7
:10255000D000D2013F30D30083128A150A126420C2
:102560008A150A12C62F8A150A12C8218A150A125C
:10257000FA228A015A2683165108EE0083128A1520
:102580000A126E22640083164008403C8A110A1623
:1025900083120319032B6400831640083B3C8A1105
:1025A0000A168312031DDD2A83162030BB00831216
:1025B0008A01A7268A110A16E32A83164008BB005F
:1025C00083128A01A72608308316A8070318A90AD0
:1025D00028088312A000831629088312A100A301F2
:1025E000EF308A0173218A110A16031DFB2A831614
:1025F0006E08D10083128A015A268A150A126E22A9
:102600008A110A16C22A8A150A12C62F8A150A12B8
:10261000C8218A150A12FA2283162808EE002A0811
:10262000EF0083128A015A268A150A126E2264006C
:1026300083164008403C8A110A16831203195C2B4A
:102640006400831640083B3C8A110A168312031D5E
:10265000322B83162030BB0083128A01A7268A11F1
:102660000A16382B83164008BB0083128A01A7265E
:1026700083166E08A800A9010830AA070318AB0A40
:102680002A088312A00083162B088312A100A3013D
:102690003F308A0173218A110A16031D542B8316B9
:1026A0006F08AA00AB0183128A015A268A150A1202
:1026B0006E228A110A16172B8A150A12C62F831644
:1026C0000230C20083128A110A16772B8316033058
:1026D000C20083128A110A16772B8316C201831255
:1026E0008A110A16772B83160130C20083128A15CD
:1026F0000A12872283164F088312F60083165008A9
:102700008312F500831652088312F80083165308CB
:102710008312F7007508F3007608F4007308A00030
:102720007408A1007808A30077088A016F218A1134
:102730000A16031D0C2C640083164208003C8A1103
:102740000A168312031DBE2B8A150A128A2107302E
:10275000BA001030B8000730BB000830B900A03014
:102760008A01202074088A01202073088A01202011
:102770007F088A011E200A308A012E2164008316F8
:102780004208013C8A110A168312031DE02B073010
:10279000BA001030B8000730BB000830B900A030D4
:1027A0008A01202074088A01202073088A012020D1
:1027B0008A0105208316C00083128A150A1274212B
:1027C000640083164208023C8A110A168312031D14
:1027D000F32B8A150A128A21730803178D0003133D
:1027E0007F088A012021640083164208033C8A1175
:1027F0000A168312031D052C73088A0118218316FB
:10280000C00083128A150A127421F30A0319F40A0C
:102810008A110A16031D8E2B8316C20183128A1594
:102820000A12C62F8A150A12872283165208AA0096
:10283000AB01831283162A088312A00083162B088B
:102840008312A1008316530883128A016E218A1114
:102850000A16031D582C83164F08A800A9018312DD
:10286000831628088312A000831629088312A1006A
:102870008316500883128A016E218A110A16031DDD
:102880004F2C8A01AA228A150A1274218316A80ADB
:102890000319A90A8A110A168312031D302C831604
:1028A000AA0A0319AB0A8A110A168312031D1A2CED
:1028B0008A150A12C62F8A150A1287228316520811
:1028C000AA00AB01831283162A088312A000831684
:1028D0002B088312A1008316530883128A016E21EC
:1028E0008A110A16031DA52C83164F08A800A901FA
:1028F0008312831628088312A000831629088312E6
:10290000A1008316500883128A016E218A110A16CB
:10291000031D9C2C8A150A128A217F088316BE008B
:1029200083128A0145278316A80A0319A90A8A1166
:102930000A168312031D792C8316AA0A0319AB0AFF
:102940008A110A168312031D632C63008A110A166A
:02295000A52CB4
:02400E00753DFE
:00000001FF
